:100000000BC0189518951895189518953FC1189517
:1000100018951895189518958FED8DBFC0ECE8EBE5
:100020004E2EDD275D2EEEE7F0E0A0E6B0E088275B
:100030008D933197E9F784B7082E877F84BF8FE1CE
:1000400081BD87E081BD662487EF8ABB8FE087BBD7
:1000500088E08BBB80E088BBE8E2F0E0A0E691E0BE
:10006000A9D3009160000D3C08F009C089EF8BBB5B
:100070008EE088BB85B78F7E806385BF8895809131
:100080006000815080936000E8E2F0E0A0E691E03B
:100090007BE77FD386E886B980E887B982E083BFB3
:1000A000789489B7826089BF82E083BFE8EAF4E090
:1000B00000D281E090E0A9E68D939C93A9E60D9192
:1000C0001C910A3050E0150710F009F00CC0F4D173
:1000D000A9E6AD90AAE6AA0D23D30C92EAD1A9E62F
:1000E000EED108F4EBCF80E08093600080E0809355
:1000F0006100A9E738D3809183008F7B80938300D0
:10010000A3E88C9187FB0EF0C0C0809183008F77AD
:100110008093830000916200003009F034C0ADE7A5
:100120000D911C9141E050E0040F151FA9E60D93BD
:100130001C93A9E6AD90AAE6AA0D8C918BBBC19841
:10014000C39AA3E88C9186FB0EF01DC0A9E70D9120
:100150001C9144E650E0DFD1A1E84D935C93A1E807
:100160000D911C9144E650E0F0D1A9E60D931C934B
:10017000A9E70D911C91A9E64D915C91041B150B0B
:10018000A5E70D931C9300916200013009F03CC07B
:10019000A3E88C9185FB0EF402C0C09A01C0C09800
:1001A000AFE70D911C9141E050E0040F151FA9E647
:1001B0000D931C93A9E6AD90AAE6AA0D8C918BBB7A
:1001C000C398C29AA3E88C9186FB0EF01DC0A5E7E8
:1001D0000D911C914AE050E09ED1AFE74D935C93A6
:1001E000AFE70D911C914AE050E0AFD1A9E60D9325
:1001F0001C93A5E70D911C91A9E64D915C91041B00
:10020000150BA7E70D931C9300916200023009F0D3
:100210003CC0A3E88C9185FB0EF002C0C09A01C0DF
:10022000C098A1E80D911C9141E050E0040F151F0A
:10023000A9E60D931C93A9E6AD90AAE6AA0D8C91B0
:100240008BBBC298C19AA3E88C9186FB0EF01DC0AF
:10025000A7E70D911C9141E050E05DD1ADE74D93D2
:100260005C93ADE70D911C9141E050E06ED1A9E6A1
:100270000D931C93A7E70D911C91A9E64D915C91FC
:10028000041B150BABE70D931C933ACF0F921F92F3
:100290002F923F924F925F927F92AF92BF920F93B5
:1002A0001F932F933F934F935F936F937F938F93FE
:1002B0009F93AF93BF93CF93DF93EF93FF938FB74A
:1002C0008F93A0E68C918F5F8C9300916000063035
:1002D00010F009F001C0CCC080E0809360008091F4
:1002E0008300806880938300A2E68C918F5F8C935B
:1002F00000916200023010F009F001C008C080E0F7
:1003000080936200809183008F7B80938300A1E6BD
:100310008C918F5F8C93009161000E3110F009F089
:1003200001C0A6C080E0809361008091830080645A
:1003300080938300CB9B09C0809183008F7D809345
:10034000830087E08093840008C0809183008062EE
:100350008093830089E180938400379A07B1007EFF
:10036000A4E88C9190E0890F082707B90AD1A3E689
:100370008D939C933798E3E6F0E0D190E080FF24E2
:1003800000275BD1A5E68AD1E2ECF7E0CDD1E5E626
:10039000F0E034D195D1EDE0A5E6EDD1A3E88C9164
:1003A00085FB0EF40BC0E6ECF7E0BED1E5E6F0E02D
:1003B00025D186D1EDE0A5E6DED154C0E5E6F0E03A
:1003C0001DD1EAECF7E0B0D1B8D108F00AC0EEECEC
:1003D000F7E0AAD1E5E6F0E011D172D1EDE0A5E6B3
:1003E000CAD1E5E6F0E00AD1EAECF7E09DD1A5D16B
:1003F00081E008F480E08F93E5E6F0E0FFD0E2EDE5
:10040000F7E092D19AD181E008F080E09F918923B2
:10041000882309F40AC0E6EDF7E086D1E5E6F0E0CE
:10042000EDD04ED1EDE0A5E6A6D1E5E6F0E0E6D0D0
:10043000E2EDF7E079D181D108F40AC0EAEDF7E006
:1004400073D1E5E6F0E0DAD03BD1EDE0A5E693D15B
:10045000EEEDF7E069D1E5E6F0E0D0D031D1EDE0A6
:10046000A5E689D1E5E6F0E095D0A9E7DD92EC922A
:100470008F918FBFFF91EF91DF91CF91BF91AF919E
:100480009F918F917F916F915F914F913F912F91AC
:100490001F910F91BF90AF907F905F904F903F90D2
:1004A0002F901F900F901895FE38DDBD3BAFEB3CB1
:1004B000FF3F8E2E9F2E0895E82DF92D0895ED9182
:1004C000FC91EF5FFF4FFC93EE93089508D03DD071
:1004D00000FC10D0089503D01ED001F8F9CF0024FD
:1004E000E89457FF02C009D0689400F80BD010F8C8
:1004F0000124089502D009D00895509540954F5F8A
:100500005F4F0895E89417FF0895009510950F5FC9
:100510001F4F68940895352F242FE894452B11F42C
:1005200068940895512F402F0027112780E1440F30
:10053000551F001F111F021B130B416018F4020FFF
:10054000131F4E7F8A9599F70895752F642F5527AD
:100550004427FF93F1E1889405C010F4460F571F1C
:100560005695479517950795FA95B9F7FF91089510
:100570003197F1F70895689462F80895E89462F865
:100580000895369A3699FECF369A3699FECF84B1C1
:1005900095B1089533D0992711278F2D880F80E8C2
:1005A000F82A802F881F08F41FEF41F08F57082F7B
:1005B00007FD04C0003240F08FEF01C08827982F5C
:1005C000D82EE82EF82E09C08FE1801B082FF69454
:1005D000E794D79497950A95D1F7112351F0909508
:1005E000D094E094F09481E0980F8827D81EE81EFC
:1005F000F81E0F2DFE2CED2CD92E0895D190E190F0
:10060000F19001910895102F90E8FF0C001F092729
:10061000990FF7941078652F90E8440F551F5927CC
:10062000990F4795607800380895FF0C90E890275F
:10063000110F9795F794092F0895102FBD2CDE2CDC
:10064000EF2CF02E11234AF4B094D094E094F0945F
:100650009FEFB91AD90AE90AF90A0EE1FF2039F425
:10066000FE2CED2CDB2CBB240850C2F723C032F04B
:100670000A95BB0CDD1CEE1CFF1CF9CF01D0D5CFB9
:10068000B7FE089590E8B91611F4D0FE08959FEFD3
:10069000D91AE90AF90A09F403950895DD92ED9251
:1006A000FD920C9308959FE7092FF92A9FEFD92E09
:1006B000E92E0895DD24EE24FF2400271127089554
:1006C000A2DFC1F35038B1F31627005850580894F0
:1006D000051F12F418F4E7CF08F0ECCF0AD0FF2082
:1006E0002AF0BB0CDD1CEE1CFF1C9FCF0F5FDBF262
:1006F0009CCF9F929924AA24BB24992788E1990C26
:10070000AA1CBB1CDD1CEE1CFF1C30F4920EA31EA9
:10071000B41ED91EE91EF91E8A9589F79F90089587
:10072000C895319600200895FBDF202DF9DF302D8C
:10073000F7DF402DF5DF502D089507FB00680EF41C
:100740000F7757FB50680EF45F7707FD02C057FF25
:1007500005C0D216E306F406050708952D153E05DB
:100760004F055007089582E001C084E099279D93CA
:100770008A95E9F7089594E081918D939A95E1F730
:100780000895E199FECFEEBB3196089591E001C046
:1007900092E07B3751F47FB7F894F3DF8D918DBBF6
:1007A000E29AE19A9A95C9F77FBF7727089591E079
:1007B00001C092E0E6DFE09A8DB38D939A95D1F770
:1007C00008951283803E3333B33F0000803F8FC2D1
:1007D000753F0000A0408716993E448B6C3E000098
:0207E0002041B6
:00000001FF
